:020000040000FA
:1000000025000400170C02000B0C060046044602F3
:100010000B0E43070D0A46040300010C3000FF0CD1
:100020002607080C0607010C6607000C3100910238
:100030004306070A11023200510C21004009070C47
:100040003400390932030307440903064209F40264
:10005000210A10023200050C34003909320303076B
:10006000440903064209F4022D0A01024307350A36
:10007000070A490C33005509F3023B0A54090008EA
:10008000620C450A300C450A180C3300040C26009B
:10009000540966004E09F302470A00080000500A9E
:1000A000510A520A0000540A0000040831083208BC
:1000B0002008620869087408200853084908520893
:1000C000430820086D0869086E0869082008490877
:1000D000520820085408720861086E0873086D08F9
:1000E0006908740874086508720820085608310801
:1000F0002E083008200868087408740870083A0848
:100100002F082F08700869086308700872086F08C4
:100110006A0865086308740873082E086F08720877
:1001200067082E0875086B08200828086308290846
:100130002008700869086308700872086F086A0868
:10014000650863087408730820083208300831080D
:04015000300820084B
:021FFE00EB0FE7
:00000001FF
